:100000002EEF07F0EA6A490EE96EEF500DE0020E9E
:10001000016E006A002EFED7012EFBD7970E006EF0
:10002000002EFED7EF2EF3D71200899A929A899864
:100030009298899692968B8894888B869496C050D5
:10004000C00B0209C06EC08EC280C150F00BC16EE1
:10005000070E0F01386F000E396F3A6F870ECD6EA5
:10006000CC6A6168F19E00017EEF07F08B8600D0BC
:1000700000D08B98949800D000D08B9600D000D000
:100080001200948800D000D08B8600D000D08B96D0
:1000900000D000D012008B98949800D000D08B86AE
:1000A00000D000D08B9600D000D01200486A485093
:1000B000060809E347AE02D0E4DF01D0ECDFD890B8
:1000C0004736482AF4D71200476A948800D000D0F7
:1000D0008B8600D000D082A808D000D000D0472A5C
:1000E0004750640801E101D0F6D78B9600D000D0CC
:1000F00000D000D08B98949800D000D0475064086E
:100100000DE1898A040E486EFA0E496E7BDF482E97
:10011000FBD7899A010E016E03D002D0000E016E4A
:1001200012008B98949800D000D08B8600D000D01D
:10013000948800D000D0120099DF43C047F0B6DFAA
:10014000AADFC2DF015204E0ECDF010E016E2BD00A
:10015000466A4650070809E344AE02D092DF01D058
:100160009ADFD8904436462AF4D7AEDF015204E035
:10017000D8DF010E016E17D0466A4650070809E322
:1001800045AE02D07EDF01D086DFD8904536462AC4
:10019000F4D79ADF015204E0C4DF010E016E03D0F0
:1001A000C0DF000E016E1200980E436E3E0E446ECC
:1001B000FE0E456EC1DF980E436E3D0E446EFE0E80
:1001C000456EBADF9A0E436E3E0E446EFE0E456ECD
:1001D000B3DF9A0E436E3D0E446EFE0E456EACDFED
:1001E0001200899A89988996346A345003081AE370
:1001F000898A89988996320E496E04DF899A89889E
:100200008996320E496EFEDE899A89988986320E69
:10021000496EF8DE899A89988996320E496EF2DE27
:10022000342AE3D7899A8998899682EF07F0346A4D
:1002300081BA01D0348081B801D0348281B601D036
:10024000348434C001F0120036C043F0446A456A79
:1002500073DF36C043F03D0E446EFE0E456E6CDF1C
:1002600036C043F03E0E446EFE0E456E65DF36C06E
:1002700043F0020E446E100E456E5EDF36C043F052
:10028000010E446E110E456E57DF36C043F03D0E31
:10029000446EFE0E456E50DF36C043F03E0E446E97
:1002A000FE0E456E49DF120036C043F0446A456ACF
:1002B00043DF36C043F03D0E446EFE0E456E3CDF1C
:1002C00036C043F03E0E446EFE0E456E35DF36C03E
:1002D00043F0030E446E456A2FDF36C043F02A0E0A
:1002E000446E110E456E28DF36C043F0020E446E98
:1002F000456A22DF36C043F00D0E446E100E456E87
:100300001BDF36C043F0250E446E080E456E14DF29
:10031000120047504902F3CF01F0F4CF00F04A0237
:10032000F350002648504902F3500020026E12009C
:1003300046C001F045C000F04566012A0900F5CF2E
:10034000EEFF002EFBD7012EF9D7F86A12003B6AA8
:1003500036C03AF03D6A37C03CF03BC048F03AC086
:1003600047F0030E4A6ED40E496ED3DF02C044F04C
:1003700001C043F03DC048F03CC047F0030E4A6E58
:10038000D40E496EC6DF02C046F001C045F002C07F
:1003900048F001C047F04A6A030E496EBADF0150C7
:1003A0004324386E02504420396E3F6A3E6A3F5003
:1003B000010837E303E13E50E80833E3200E382418
:1003C000436EA40E3920446EF86AF76E43C0F6FF00
:1003D000EA6A410EE96E466A010E456EA9DF382AC7
:1003E000D8B4392A200E3824436EA40E3920446E26
:1003F000F86AF76E43C0F6FFEA6A420EE96E466A93
:10040000010E456E95DF382AD8B4392A9A0E436E0C
:1004100041C044F042C045F08FDE3E2AD8B43F2AA6
:10042000C6D71200980E366E0FDF9A0E366E0CDFAE
:10043000980E366E39DF9A0E366E36DF050E496E2F
:10044000E1DD34501BE0010A19E0030A17E0010A5C
:1004500015E0070A13E0010A11E0030A14E0010A9B
:1004600012E00F0A16E0010A14E0030A12E0010A82
:1004700010E0070A0EE0010A0CE011D0366A04C051
:1004800037F065DF10D0010E366E04C037F05FDF45
:100490000AD0020E366E04C037F059DF04D0366A37
:1004A00004C037F054DF1200CF6ACE6A050E496EE1
:1004B000A9DDCE50346ECFCF35F0366A355203E128
:1004C00034504B0808E2355206E13450530803E338
:1004D000010E366EC3D0355203E13450680808E28D
:1004E000355206E13450720803E3020E366EB6D080
:1004F000355203E13450980808E2355206E1345091
:10050000A60803E3030E366EA9D0355203E134503A
:10051000D20808E2355206E13450E50803E3040E40
:10052000366E9CD0355203E13450E50808E235526E
:1005300006E13450F90803E3050E366E8FD03550CE
:1005400000080FE2FF0A03E13450A6080AE2355022
:10055000010807E303E13450CA0803E3060E366ED0
:100560007DD0355000080FE2FF0A03E13450CB087C
:100570000AE23550010807E303E13450F30803E3CE
:10058000070E366E6BD0355002080FE2FF0A03E10A
:1005900034504D080AE23550030807E303E13450B4
:1005A000950803E3080E366E59D0355002080FE265
:1005B000FF0A03E1345098080AE23550030807E3C4
:1005C00003E13450E60803E3090E366E47D0355098
:1005D00005080FE2FF0A03E134509C080AE2355097
:1005E000070807E303E134502A0803E30A0E366ED6
:1005F00035D0355006080FE2FF0A03E134503208C7
:100600000AE23550070807E303E13450CC0803E35E
:100610000B0E366E23D035500C080FE2FF0A03E1B3
:10062000345039080AE235500E0807E303E134502C
:10063000550803E30C0E366E11D035500D080EE24E
:10064000FF0A03E13450650809E235500F0806E35C
:1006500003E13450990802E30D0E366E36C001F006
:10066000B1EF07F03450010A19E0030A17E0010A5C
:1006700015E0070A13E0010A11E0030A12E0010A7B
:1006800010E00F0A11E0010A0FE0030A10E0010A6E
:100690000EE0070A19E0010A17E023D0898889963D
:1006A00022D0899889861FD0898889861CD02C50B1
:1006B000270802E3899801D0898889962C2A2C5032
:1006C000500801E12C6A0FD02C50270802E38996CC
:1006D00001D0898689982C2A2C50500801E12C6A77
:1006E00002D089988996B7EF07F0C2824290C2A2E1
:1006F000428042B004D04290C2A24280FAD7C2B235
:10070000FED7C4CF03F0C3CF43F0C4CF44F043C0FF
:1007100001F044C002F0A2EF03F03E34006E003658
:10072000FC0E0016C250830B0010C26E1A0E006E33
:10073000002EFED70000406A3F6A416A41500F0810
:1007400009E3D3D702C003F001503F2603504022F3
:10075000412AF4D740323F3240323F3240323F32BA
:1007600040323F320F0E40163FC001F040C002F051
:1007700012001C5226E03B6A3B50040821E3D8904B
:100780003B34036A1D0F016E000E032201C03CF0D2
:1007900003C03DF038C03EF0C0DF3DC0EAFF3CC0C2
:1007A000E9FF02C0ECFFED5201C0EFFF036A3B50CE
:1007B000270FE96E000E0320EA6EEF6A3B2ADCD7B2
:1007C0001C6A38C03EF0A9DF02C03AF001C039F01F
:1007D000036A3850270FE96E000E0320EA6EEF2CF3
:1007E00052D0D8903834036A1D0FE96E000E0320F2
:1007F000EA6EECCF3DF0ED52EFCF3CF03D503A5C6D
:1008000012E303E139503C5C0EE2D8903834036ABD
:100810001D0FE96E000E0320EA6E3AC0ECFFED52A8
:1008200039C0EFFF2FD0D8903834036A1D0FE96E1E
:10083000000E0320EA6EECCF3DF0ED52EFCF3CF01E
:10084000010E3924016E000E3A20036E03503D5C08
:1008500019E303E13C50015C15E2D8903834036A97
:100860001D0FE96E000E0320EA6E3AC0ECFFED5258
:1008700039C0EFFF036A3850270FE96E000E0320DE
:10088000EA6EEF6A50D0D8903834036A1D0FE96ED3
:10089000000E0320EA6EECCF3DF0ED52EFCF3CF0BE
:1008A0003A503D5C12E303E13C50395C0EE2D890D3
:1008B0003834036A1D0FE96E000E0320EA6E3AC059
:1008C000ECFFED5239C0EFFF2ED0D8903834036AD8
:1008D0001D0FE96E000E0320EA6EECCF3DF0ED52E5
:1008E000EFCF3CF0010E3C26000E3D223D503A5C1D
:1008F0001AE303E139503C5C16E2D8903834036ABD
:100900001D0FE96E000E0320EA6E3AC0ECFFED52B7
:1009100039C0EFFF036A3850270FE96E000E03203D
:10092000EA6E010EEF6ED8903834036A1D0FE96E3F
:10093000000E0320EA6EEFCF01F0EE52EDCF02F091
:100940001200395001082EE303E1385000082AE371
:1009500039C048F038C047F04A6A3F0E496ED9DCCA
:1009600002C03BF001C03AF03B323A323B323A32FD
:100970003B323A323B323A323B323A323B323A3213
:100980003B323A32010E3B163A1C3D6E3B1C3E6E2A
:100990003D2AD8B43E2AFE0E3D243A6E000E3E207B
:1009A0003B6E5AD0395001082BE3000E385C3D6E87
:1009B000010E39583E6E486E3DC047F04A6A050E3A
:1009C000496EA7DC02C03BF001C03AF03B323A323C
:1009D0003B323A323B323A323B323A323B323A32B3
:1009E000070E3B163A1C3D6E3B1C3E6E3D2AD8B4AA
:1009F0003E2A800E3D243A6E000E3E203B6E2CD0E7
:100A0000000E385C3D6E020E39583E6E486E3DC099
:100A100047F04A6A050E496E7CDC02C03BF001C01B
:100A20003AF03B323A323B323A323B323A323B32A4
:100A30003A323B323A323B323A32030E3B163A1CE0
:100A40003D6E3B1C3E6E3D2AD8B43E2A580E3D24D6
:100A50003A6E000E3E203B6E3A3C05D03B5203E11D
:100A60003B6AFE0E3A6E3AC03CF03AC001F056EFD7
:100A700006F0016A026A006A036A445002E14350C8
:100A800018E0100E456ED8904136423600360336D7
:100A90004450035C02E14350005C07E34350005EB6
:100AA000D8A003064450035ED88001360236452E96
:100AB000EAD712003D6A3C6A3B5001082AE2FF0A6D
:100AC00003E13A501C0825E281A412D01C0E3A5CC6
:100AD0003F6E020E3B58406E426E3FC041F0446A8A
:100AE000150E436EC6DF02C03DF001C03CF011D0D0
:100AF0001C0E3A5C3F6E020E3B58406E426E3FC089
:100B000041F0446A0C0E436EB4DF02C03DF001C0F8
:100B10003CF03CC03EF03EC001F012003D6A3C6A31
:100B20003B5001082BE303E13A50DF0827E381A49F
:100B300013D0E00ED8803A543F6E010E3B54406E05
:100B4000426E3FC041F0446A150E436E92DF02C010
:100B50003DF001C03CF012D0E00ED8803A543F6E18
:100B6000010E3B54406E426E3FC041F0446A0C0E91
:100B7000436E7FDF02C03DF001C03CF03CC03EF060
:100B80003EC001F0120094888B8600D000D082A86D
:100B900003D0010E3C6E01D03C6A8B9600D000D091
:100BA0003CC001F01EEF06F036EC00F038C047F014
:100BB00056EC00F04BEC00F064EC00F0015205E064
:100BC00091EC00F0010E016E4BD03A6A3A500708E2
:100BD0000BE339AE03D041EC00F002D04BEC00F057
:100BE000D89039363A2AF2D78B8600D000D0948834
:100BF00000D000D08B9600D000D08B8600D000D0E3
:100C00008B98949800D000D08B9600D000D038C03C
:100C100047F056EC00F041EC00F064EC00F00152BB
:100C200005E091EC00F0010E016E1AD03B6A3A6AC1
:100C30003A50070808E3D8903B36A5D7015201E0A7
:100C40003B803A2AF5D7948800D000D08B8600D01C
:100C500000D08B9600D000D091EC00F03BC001F0AA
:100C60001200386A86DD02C006F001C005F081B2CC
:100C700008D0010E386E7DDD02C00AF001C009F017
:100C800003D0020E0A6E096A81B008D0020E386ED7
:100C900070DD02C008F001C007F003D0020E086E3C
:100CA000076A06C039F005C038F04BD601C034F0F1
:100CB000396A34C038F008C03BF007C03AF0FADEB9
:100CC000036A01503826035039220AC03BF009C09C
:100CD0003AF024DF036A01503824366E035039207D
:100CE000376E375203E13650FD0803E2376AFE0ED5
:100CF000366E36C00BF0396A34C038F008C03BF0AD
:100D000007C03AF00BDF036A01503826035039223E
:100D10000AC03BF009C03AF001DF036A01503824F1
:100D2000366E03503920376E375203E13650FD08D6
:100D300003E2376AFE0E366E36C00CF0396A34C0F4
:100D400038F008C03BF007C03AF0B4DE036A015047
:100D50003826035039220AC03BF009C03AF0AADE17
:100D6000036A01503824366E03503920376E3752EB
:100D700003E13650FD0803E2376AFE0E366E36C0D8
:100D80000DF0396A34C038F008C03BF007C03AF0C3
:100D9000C5DE036A01503826035039220AC03BF0F1
:100DA00009C03AF087DE036A01503824366E0350DA
:100DB0003920376E375203E13650FD0803E2376AB7
:100DC000FE0E366E36C00EF0980E386E3E0E396E40
:100DD000EBDE01C035F00B50355C08E0980E436E39
:100DE0003E0E446E0BC045F09CEC00F0980E386E41
:100DF0003D0E396ED9DE01C035F00C50355C08E08F
:100E0000980E436E3D0E446E0CC045F09CEC00F015
:100E10009A0E386E3E0E396EC7DE01C035F00D50A9
:100E2000355C08E09A0E436E3E0E446E0DC045F0F0
:100E30009CEC00F09A0E386E3D0E396EB5DE01C0A6
:100E400035F00E50355C08E09A0E436E3D0E446E50
:100E50000EC045F09CEC00F0C8EF07F0F86AD09E99
:100E6000600ED36E9B9C9B9E010E0F6E1C6E2C6AB7
:100E70000F01386B396B3A6B776A786A796A05D0FB
:100E80000C4010000F401D000000000EF86E0E0E0A
:100E9000F76E800EF66E0900F550006E000A13E042
:100EA0000900F550016EE8BE05D00F0BEA6E09008F
:100EB000F5CFE9FF01BC090001AC0900F5CFEEFF59
:100EC000004EE9D7F9D7F86A040E346EFA0E496E6F
:100ED000000102EC00F0342E01D002D00F01F6D751
:100EE000FF0E926E936E946E600ED36E9B9C9B9ED3
:100EF000640E496E02EC00F015EF00F0D4EC00F047
:100F0000F1EF00F089988996D4EC00F017EC01F02D
:100F100001C004F0346A12EC02F0010E2D6E2F6A4B
:100F20002FC02EF02D5211E082B40FD017EC01F03B
:100F300001C004F0D4EC00F02EC034F012EC02F04A
:100F40002D6A050E496E02EC00F02D5208E182A4D4
:100F500006D0010E2D6E050E496E02EC00F054EF26
:100F600002F001C02EF02EC034F032EF03F02F500B
:100F70002E5C08E02E5204E02EC034F012EC02F099
:100F80002EC02FF02E5202E06CD602D0D4EC00F02E
:040F9000C9D70300BA
:10A42000000000010304000003110210002C0800CA
:10A4300009000ADA0B000C000D000EDA0F00100004
:10A44000110012DA1300147F153716BB170018819C
:10A45000198C1AEC1B001C7F1DFF1EFF1F00200023
:10A4600021002200230024002500260027002800C8
:10A4700029002A002B002C002D002E002F00304038
:10A48000310032003300344035003600370038FFE9
:10A4900039FF3AFF3B003C803D003E003F0040401A
:10A4A000410042004300447F45FF46FF470048000B
:10A4B00049004A004B004C034DC04E004F00500B6A
:10A4C000514052005300003E080009000ADA0B0018
:10A4D0000C000D000EDA0F001000110012DA13004C
:10A4E000147F153716BB17001881198C1AEC1B0046
:10A4F0001C7F1DFF1EFF1F002000210022002300E3
:10A500002400250026002700280029002A002B000F
:10A510002C002D002E002F0030403100320033007F
:10A52000344035003600370038FF39FF3AFF3B0032
:10A530003C803D003E003F0040404100420043005F
:10A54000447F45FF46FF4700480049004A004B0052
:10A550004C034DC04E004F00500B51405200530071
:10A560000098080009000A000B000C000D000E0006
:10A570000F00100011101200130014001510160423
:10A580001701180019601A281B001C001D701E2CD2
:10A590001F012000210022002300240025002600A6
:10A5A0002700280029402A002B022C002D602E387D
:10A5B0002F023000316032083305340135B03604E3
:10A5C0003704380039403A043B033C003D703E00FC
:10A5D0003F03400141B0420C430744004570461020
:10A5E0004708480049004A004B004C004D004E000F
:10A5F0004F005000514052005306540055605638E9
:10A600005706580059605A1C5B0B5C015DB05E1820
:10A610005F0A60006140620463096400657066144B
:10A620006709680169B06A206B0D6C006D706E245B
:10A630006F0E700071007200730074007500760078
:10A640007700780079407A007B0C7C007D607E3852
:10A650007F0C0099080009600A380B0C0C000D00F3
:10A660000E000F00100011401204131814001540C2
:10A6700016041736180019601A471BFB1C001D0032
:10A680001E001F002000210022002300240025308E
:10A6900026F02702280129142A832B772C002D006D
:10A6A0002E002F0030003160324B33FB3400350078
:10A6B00036003700380039003A003B003C003D309E
:10A6C0003EF03F024001411442834377440045007D
:10A6D000460047004800496F4AEC4B0F4C004D6F55
:10A6E0004EEC4F1050005130520053025400553080
:10A6F000560057025800596F5AEC5B115C005D6FB1
:10A700005EEC5F12600061306200630264006530DD
:10A71000660067026800696F6AEC6B136C006D6F0E
:10A720006EEC6F147000713072007302740075303B
:10A73000760077027800796F7AEC7B157C007D6F6C
:10A740007EEC7F16009A080009300A000B020C000C
:10A750000D300E000F021000116F12F0132D1400B7
:10A76000156F16F0172E180019301A041B021C0062
:10A770001D301E041F022000216F22F0232F240011
:10A78000256F26F02730280029302A042B022C00C0
:10A790002D302E042F023000316F32F0333134006F
:10A7A000356F36F03732380039303A043B023C001E
:10A7B0003D303E043F024000416F42F043334400CD
:10A7C000456F46F04734480049304A044B024C007C
:10A7D0004D304E044F0250015110520353FF000000
:10A7E0002B1F002C04000104000002000804530782
:10A7F0000300FFFF0000000103040000031102102A
:10A80000002C080009000A2E0B000C000D000E2E73
:10A810000F0010001100122E1300147F15A416252E
:10A820001700188019B61AF11B001C7F1DFF1EFFB0
:10A830001F00200021002200230024002500260004
:10A840002700280029002A002B002C002D002E00B4
:10A850002F003040310032003300344035003600E4
:10A86000370038FF39FF3AFF3B003C803D003E0097
:10A870003F004040410042004300447F45FF46FF07
:10A880004700480049004A004B004C034DC04E00B1
:10A890004F00500B514052005300003E0800090089
:10A8A0000A2E0B000C000D000E2E0F0010001100E0
:10A8B000122E1300147F15A416251700188019B640
:10A8C0001AF11B001C7F1DFF1EFF1F00200021002E
:10A8D000220023002400250026002700280029004C
:10A8E0002A002B002C002D002E002F0030403100BC
:10A8F00032003300344035003600370038FF39FF6E
:10A900003AFF3B003C803D003E003F00404041009C
:10A9100042004300447F45FF46FF4700480049008E
:10A920004A004B004C034DC04E004F00500B5140AD
:10A93000520053000098080009000A000B000C00A8
:10A940000D000E000F001000111012001300140073
:10A95000151016041701180019601A281B001C0096
:10A960001D701E2C1F012000210022002300240046
:10A97000250026002700280029402A002B022C0051
:10A980002D602E382F02300031603208330534013B
:10A9900035B036043704380039403A043B033C00F4
:10A9A0003D703E003F03400141B0420C430744006C
:10A9B000457046104708480049004A004B004C00CB
:10A9C0004D004E004F0050005140520053065400BD
:10A9D000556056385706580059605A1C5B0B5C018D
:10A9E0005DB05E185F0A6000614062046309640044
:10A9F000657066146709680169B06A206B0D6C00A8
:10AA00006D706E246F0E7000710072007300740020
:10AA1000750076007700780079407A007B0C7C0026
:10AA20007D607E387F0C0099080009600A380B0CA5
:10AA30000C000D000E000F0010001140120413183E
:10AA40001400154016041736180019601A471BFB2E
:10AA50001C001D001E001F002000210022002300FA
:10AA60002400253026F02702280129142A832B7779
:10AA70002C002D002E002F0030003160324B33FBB4
:10AA80003400350036003700380039003A003B000A
:10AA90003C003D303EF03F02400141144283437789
:10AAA00044004500460047004800496F4AEC4B0F00
:10AAB0004C004D6F4EEC4F1050005130520053027D
:10AAC00054005530560057025800596F5AEC5B112C
:10AAD0005C005D6F5EEC5F126000613062006302DB
:10AAE00064006530660067026800696F6AEC6B138A
:10AAF0006C006D6F6EEC6F14700071307200730239
:10AB000074007530760077027800796F7AEC7B15E7
:10AB10007C007D6F7EEC7F16009A080009300A00E9
:10AB20000B020C000D300E000F021000116F12F01E
:10AB3000132D1400156F16F0172E180019301A0473
:10AB40001B021C001D301E041F022000216F22F07A
:10AB5000232F2400256F26F02730280029302A04CF
:10AB60002B022C002D302E042F023000316F32F0DA
:10AB700033313400356F36F03732380039303A042B
:10AB80003B023C003D303E043F024000416F42F03A
:10AB900043334400456F46F04734480049304A0487
:10ABA0004B024C004D304E044F02500151105203E5
:10ABB00053FF00002B1F002C0400010400000200C2
:10ABC000080453070300FFFF000000010304000016
:10ABD00003110210002C080009000A0B0B000C00E6
:10ABE0000D000E0B0F0010001100120B1300147F4C
:10ABF00015D2161A17001880195B1A9A1B001C7FB1
:10AC00001DFF1EFF1F002000210022002300240042
:10AC1000250026002700280029002A002B002C00F0
:10AC20002D002E002F003040310032003300344020
:10AC300035003600370038FF39FF3AFF3B003C80D3
:10AC40003D003E003F004040410042004300447F41
:10AC500045FF46FF4700480049004A004B004C03AF
:10AC60004DC04E004F00500B514052005300003E6B
:10AC7000080009000A0B0B000C000D000E0B0F0062
:10AC800010001100120B1300147F15D2161A1700B2
:10AC90001880195B1A9A1B001C7F1DFF1EFF1F00E6
:10ACA0002000210022002300240025002600270088
:10ACB000280029002A002B002C002D002E002F0038
:10ACC0003040310032003300344035003600370068
:10ACD00038FF39FF3AFF3B003C803D003E003F001B
:10ACE0004040410042004300447F45FF46FF47008B
:10ACF000480049004A004B004C034DC04E004F0035
:10AD0000500B5140520053000098080009000A00FF
:10AD10000B000C000D000E000F00100011101200AF
:10AD200013001400151016041701180019601A28D2
:10AD30001B001C001D701E2C1F0120002100220082
:10AD400023002400250026002700280029402A008F
:10AD50002B022C002D602E382F023000316032087B
:10AD60003305340135B036043704380039403A042D
:10AD70003B033C003D703E003F03400141B0420CAC
:10AD800043074400457046104708480049004A0000
:10AD90004B004C004D004E004F00500051405200FF
:10ADA00053065400556056385706580059605A1CCF
:10ADB0005B0B5C015DB05E185F0A6000614062047D
:10ADC00063096400657066146709680169B06A20E8
:10ADD0006B0D6C006D706E246F0E70007100720050
:10ADE00073007400750076007700780079407A006F
:10ADF0007B0C7C007D607E387F0C00990800096028
:10AE00000A380B0C0C000D000E000F001000114052
:10AE10001204131814001540160417361800196090
:10AE20001A471BFB1C001D001E001F0020002100F4
:10AE3000220023002400253026F0270228012914AF
:10AE40002A832B772C002D002E002F00300031603C
:10AE5000324B33FB34003500360037003800390000
:10AE60003A003B003C003D303EF03F0240014114BF
:10AE70004283437744004500460047004800496F3D
:10AE80004AEC4B0F4C004D6F4EEC4F1050005130C0
:10AE90005200530254005530560057025800596F63
:10AEA0005AEC5B115C005D6F5EEC5F12600061301C
:10AEB0006200630264006530660067026800696FC3
:10AEC0006AEC6B136C006D6F6EEC6F147000713078
:10AED0007200730274007530760077027800796F23
:10AEE0007AEC7B157C007D6F7EEC7F16009A080063
:10AEF00009300A000B020C000D300E000F0210008A
:10AF0000116F12F0132D1400156F16F0172E180084
:10AF100019301A041B021C001D301E041F022000E1
:10AF2000216F22F0232F2400256F26F027302800E0
:10AF300029302A042B022C002D302E042F02300041
:10AF4000316F32F033313400356F36F0373238003C
:10AF500039303A043B023C003D303E043F024000A1
:10AF6000416F42F043334400456F46F04734480098
:10AF700049304A044B024C004D304E044F02500100
:10AF80005110520353FF00002B1F002C040001043A
:10AF900000000200080453070300FFFF0000000147
:10AFA0000304000003110210002C080009010A82AA
:10AFB0000B000C000D010E820F0010001101128217
:10AFC0001300147E15F416B81700188219101A27EA
:10AFD0001B001C001D011E821F0020002101228277
:10AFE00023002400250126822700287E29F42AB880
:10AFF0002B002C822D102E272F00304031003200E4
:10B000003300344035003600370038FF39FF3AFF4F
:10B010003B003C803D003E003F004040410042007C
:10B020004300447F45FF46FF4700480049004A006F
:10B030004B004C034DC04E004F00500B514052008E
:10B040005300003E080009010A820B000C000D01AC
:10B050000E820F001000110112821300147E15F4ED
:10B0600016B81700188219101A271B001C001D01A2
:10B070001E821F00200021012282230024002501BE
:10B0800026822700287E29F42AB82B002C822D1036
:10B090002E272F003040310032003300344035007D
:10B0A0003600370038FF39FF3AFF3B003C803D0057
:10B0B0003E003F004040410042004300447F45FFC6
:10B0C00046FF4700480049004A004B004C034DC072
:10B0D0004E004F00500B51405200530000980800A2
:10B0E00009000A000B000C000D000E000F001000FC
:10B0F0001110120013001400151016041701180087
:10B1000019601A281B001C001D701E2C1F01200036
:10B11000210022002300240025002600270028000B
:10B1200029402A002B022C002D602E382F023000DF
:10B13000316032083305340135B036043704380045
:10B1400039403A043B033C003D703E003F03400160
:10B1500041B0420C43074400457046104708480080
:10B1600049004A004B004C004D004E004F0050007B
:10B170005140520053065400556056385706580047
:10B1800059605A1C5B0B5C015DB05E185F0A600081
:10B1900061406204630964006570661467096801B0
:10B1A00069B06A206B0D6C006D706E246F0E7000BC
:10B1B00071007200730074007500760077007800EB
:10B1C00079407A007B0C7C007D607E387F0C009992
:10B1D000080009600A380B0C0C000D000E000F006F
:10B1E00010001140120413181400154016041736ED
:10B1F000180019601A471BFB1C001D001E001F00D1
:10B2000020002100220023002400253026F0270200
:10B21000280129142A832B772C002D002E002F00C3
:10B2200030003160324B33FB3400350036003700DC
:10B23000380039003A003B003C003D303EF03F0210
:10B2400040014114428343774400450046004700D3
:10B250004800496F4AEC4B0F4C004D6F4EEC4F10BD
:10B2600050005130520053025400553056005702DE
:10B270005800596F5AEC5B115C005D6F5EEC5F1219
:10B28000600061306200630264006530660067023E
:10B290006800696F6AEC6B136C006D6F6EEC6F1475
:10B2A000700071307200730274007530760077029E
:10B2B0007800796F7AEC7B157C007D6F7EEC7F16D1
:10B2C000009A080009300A000B020C000D300E0035
:10B2D0000F021000116F12F0132D1400156F16F0ED
:10B2E000172E180019301A041B021C001D301E04F2
:10B2F0001F022000216F22F0232F2400256F26F04B
:10B300002730280029302A042B022C002D302E044F
:10B310002F023000316F32F033313400356F36F0A8
:10B320003732380039303A043B023C003D303E04AD
:10B330003F024000416F42F043334400456F46F006
:10B340004734480049304A044B024C004D304E040B
:10B350004F0250015110520353FF00002B1F002CCD
:10B360000400010400000200080453070300FFFF6B
:10B37000000000010304000003110210002C08006B
:10B3800009000A510B000C000D000E510F001000B7
:10B39000110012511300147F1585167917001880BB
:10B3A00019F31AB11B001C001D001E511F002000C4
:10B3B0002100225123002400250026512700287F48
:10B3C00029852A792B002C802DF32EB12F003040B7
:10B3D000310032003300344035003600370038FF8A
:10B3E00039FF3AFF3B003C803D003E003F004040BB
:10B3F000410042004300447F45FF46FF47004800AC
:10B4000049004A004B004C034DC04E004F00500B0A
:10B41000514052005300003E080009000A510B0041
:10B420000C000D000E510F001000110012511300FE
:10B43000147F158516791700188019F31AB11B00AF
:10B440001C001D001E511F0020002100225123005E
:10B450002400250026512700287F29852A792B00E2
:10B460002C802DF32EB12F003040310032003300FC
:10B47000344035003600370038FF39FF3AFF3B00D3
:10B480003C803D003E003F00404041004200430000
:10B49000447F45FF46FF4700480049004A004B00F3
:10B4A0004C034DC04E004F00500B51405200530012
:10B4B0000098080009000A000B000C000D000E00A7
:10B4C0000F001000111012001300140015101604C4
:10B4D0001701180019601A281B001C001D701E2C73
:10B4E0001F01200021002200230024002500260047
:10B4F0002700280029402A002B022C002D602E381E
:10B500002F023000316032083305340135B0360483
:10B510003704380039403A043B033C003D703E009C
:10B520003F03400141B0420C4307440045704610C0
:10B530004708480049004A004B004C004D004E00AF
:10B540004F00500051405200530654005560563889
:10B550005706580059605A1C5B0B5C015DB05E18C1
:10B560005F0A6000614062046309640065706614EC
:10B570006709680169B06A206B0D6C006D706E24FC
:10B580006F0E700071007200730074007500760019
:10B590007700780079407A007B0C7C007D607E38F3
:10B5A0007F0C0099080009600A380B0C0C000D0094
:10B5B0000E000F0010001140120413181400154063
:10B5C00016041736180019601A471BFB1C001D00D3
:10B5D0001E001F002000210022002300240025302F
:10B5E00026F02702280129142A832B772C002D000E
:10B5F0002E002F0030003160324B33FB3400350019
:10B6000036003700380039003A003B003C003D303E
:10B610003EF03F024001411442834377440045001D
:10B62000460047004800496F4AEC4B0F4C004D6FF5
:10B630004EEC4F1050005130520053025400553020
:10B64000560057025800596F5AEC5B115C005D6F51
:10B650005EEC5F126000613062006302640065307E
:10B66000660067026800696F6AEC6B136C006D6FAF
:10B670006EEC6F14700071307200730274007530DC
:10B68000760077027800796F7AEC7B157C007D6F0D
:10B690007EEC7F16009A080009300A000B020C00AD
:10B6A0000D300E000F021000116F12F0132D140058
:10B6B000156F16F0172E180019301A041B021C0003
:10B6C0001D301E041F022000216F22F0232F2400B2
:10B6D000256F26F02730280029302A042B022C0061
:10B6E0002D302E042F023000316F32F03331340010
:10B6F000356F36F03732380039303A043B023C00BF
:10B700003D303E043F024000416F42F0433344006D
:10B71000456F46F04734480049304A044B024C001C
:10B720004D304E044F0250015110520353FF0000A0
:10B730002B1F002C04000104000002000804530722
:10B740000300FFFF000000010304000003110210CA
:10B75000002C080009000A140B000C000D000E1448
:10B760000F001000110012141300147F15C216CA26
:10B7700017001880197A1A141B001C001D001E14D3
:10B780001F0020002100221423002400250026147D
:10B790002700287F29C22ACA2B002C802D7A2E143C
:10B7A0002F00304031003200330034403500360085
:10B7B000370038FF39FF3AFF3B003C803D003E0038
:10B7C0003F004040410042004300447F45FF46FFA8
:10B7D0004700480049004A004B004C034DC04E0052
:10B7E0004F00500B514052005300003E080009002A
:10B7F0000A140B000C000D000E140F0010001100B5
:10B8000012141300147F15C216CA17001880197A73
:10B810001A141B001C001D001E141F002000210014
:10B82000221423002400250026142700287F29C283
:10B830002ACA2B002C802D7A2E142F003040310084
:10B8400032003300344035003600370038FF39FF0E
:10B850003AFF3B003C803D003E003F00404041003D
:10B8600042004300447F45FF46FF4700480049002F
:10B870004A004B004C034DC04E004F00500B51404E
:10B88000520053000098080009000A000B000C0049
:10B890000D000E000F001000111012001300140014
:10B8A000151016041701180019601A281B001C0037
:10B8B0001D701E2C1F0120002100220023002400E7
:10B8C000250026002700280029402A002B022C00F2
:10B8D0002D602E382F0230003160320833053401DC
:10B8E00035B036043704380039403A043B033C0095
:10B8F0003D703E003F03400141B0420C430744000D
:10B90000457046104708480049004A004B004C006B
:10B910004D004E004F00500051405200530654005D
:10B92000556056385706580059605A1C5B0B5C012D
:10B930005DB05E185F0A60006140620463096400E4
:10B94000657066146709680169B06A206B0D6C0048
:10B950006D706E246F0E70007100720073007400C1
:10B96000750076007700780079407A007B0C7C00C7
:10B970007D607E387F0C0099080009600A380B0C46
:10B980000C000D000E000F001000114012041318DF
:10B990001400154016041736180019601A471BFBCF
:10B9A0001C001D001E001F0020002100220023009B
:10B9B0002400253026F02702280129142A832B771A
:10B9C0002C002D002E002F0030003160324B33FB55
:10B9D0003400350036003700380039003A003B00AB
:10B9E0003C003D303EF03F0240014114428343772A
:10B9F00044004500460047004800496F4AEC4B0FA1
:10BA00004C004D6F4EEC4F1050005130520053021D
:10BA100054005530560057025800596F5AEC5B11CC
:10BA20005C005D6F5EEC5F1260006130620063027B
:10BA300064006530660067026800696F6AEC6B132A
:10BA40006C006D6F6EEC6F147000713072007302D9
:10BA500074007530760077027800796F7AEC7B1588
:10BA60007C007D6F7EEC7F16009A080009300A008A
:10BA70000B020C000D300E000F021000116F12F0BF
:10BA8000132D1400156F16F0172E180019301A0414
:10BA90001B021C001D301E041F022000216F22F01B
:10BAA000232F2400256F26F02730280029302A0470
:10BAB0002B022C002D302E042F023000316F32F07B
:10BAC00033313400356F36F03732380039303A04CC
:10BAD0003B023C003D303E043F024000416F42F0DB
:10BAE00043334400456F46F04734480049304A0428
:10BAF0004B024C004D304E044F0250015110520386
:10BB000053FF00002B1F002C040001040000020062
:10BB1000080453070300FFFF0000000103040000B6
:10BB200003110210002C080009020A5B0B000C0034
:10BB30000D020E5B0F0010001102125B1300147E49
:10BB400015B116951700188219921AD91B001C00FE
:10BB50001D021E5B1F0020002102225B2300240027
:10BB60002502265B2700287E29B12A952B002C82EE
:10BB70002D922ED92F003040310032003300344056
:10BB800035003600370038FF39FF3AFF3B003C8074
:10BB90003D003E003F004040410042004300447FE2
:10BBA00045FF46FF4700480049004A004B004C0350
:10BBB0004DC04E004F00500B514052005300003E0C
:10BBC000080009020A5B0B000C000D020E5B0F005F
:10BBD00010001102125B1300147E15B116951700A8
:10BBE000188219921AD91B001C001D021E5B1F002F
:10BBF00020002102225B230024002502265B27006F
:10BC0000287E29B12A952B002C822D922ED92F0027
:10BC10003040310032003300344035003600370008
:10BC200038FF39FF3AFF3B003C803D003E003F00BB
:10BC30004040410042004300447F45FF46FF47002B
:10BC4000480049004A004B004C034DC04E004F00D5
:10BC5000500B5140520053000098080009000A00A0
:10BC60000B000C000D000E000F0010001110120050
:10BC700013001400151016041701180019601A2873
:10BC80001B001C001D701E2C1F0120002100220023
:10BC900023002400250026002700280029402A0030
:10BCA0002B022C002D602E382F023000316032081C
:10BCB0003305340135B036043704380039403A04CE
:10BCC0003B033C003D703E003F03400141B0420C4D
:10BCD00043074400457046104708480049004A00A1
:10BCE0004B004C004D004E004F00500051405200A0
:10BCF00053065400556056385706580059605A1C70
:10BD00005B0B5C015DB05E185F0A6000614062041D
:10BD100063096400657066146709680169B06A2088
:10BD20006B0D6C006D706E246F0E700071007200F0
:10BD300073007400750076007700780079407A000F
:10BD40007B0C7C007D607E387F0C009908000960C8
:10BD50000A380B0C0C000D000E000F0010001140F3
:10BD60001204131814001540160417361800196031
:10BD70001A471BFB1C001D001E001F002000210095
:10BD8000220023002400253026F027022801291450
:10BD90002A832B772C002D002E002F0030003160DD
:10BDA000324B33FB340035003600370038003900A1
:10BDB0003A003B003C003D303EF03F024001411460
:10BDC0004283437744004500460047004800496FDE
:10BDD0004AEC4B0F4C004D6F4EEC4F105000513061
:10BDE0005200530254005530560057025800596F04
:10BDF0005AEC5B115C005D6F5EEC5F1260006130BD
:10BE00006200630264006530660067026800696F63
:10BE10006AEC6B136C006D6F6EEC6F147000713018
:10BE20007200730274007530760077027800796FC3
:10BE30007AEC7B157C007D6F7EEC7F16009A080003
:10BE400009300A000B020C000D300E000F0210002A
:10BE5000116F12F0132D1400156F16F0172E180025
:10BE600019301A041B021C001D301E041F02200082
:10BE7000216F22F0232F2400256F26F02730280081
:10BE800029302A042B022C002D302E042F023000E2
:10BE9000316F32F033313400356F36F037323800DD
:10BEA00039303A043B023C003D303E043F02400042
:10BEB000416F42F043334400456F46F04734480039
:10BEC00049304A044B024C004D304E044F025001A1
:10BED0005110520353FF00002B1F002C04000104DB
:10BEE00000000200080453070300FFFF00000001E8
:10BEF0000304000003110210002C080009000A7F4F
:10BF00000B000C000D000E7F0F0010001100127FBF
:10BF10001300147F156616C61700188119301A55BC
:10BF20001B001C001D001E7F1F0020002100227F1F
:10BF3000230024002500267F2700287F29662AC6A3
:10BF40002B002C812D302E552F0030403100320037
:10BF50003300344035003600370038FF39FF3AFFF0
:10BF60003B003C803D003E003F004040410042001D
:10BF70004300447F45FF46FF4700480049004A0010
:10BF80004B004C034DC04E004F00500B514052002F
:10BF90005300003E080009000A7F0B000C000D0052
:10BFA0000E7F0F0010001100127F1300147F156622
:10BFB00016C61700188119301A551B001C001D00E9
:10BFC0001E7F1F0020002100227F23002400250067
:10BFD000267F2700287F29662AC62B002C812D303A
:10BFE0002E552F00304031003200330034403500F0
:10BFF0003600370038FF39FF3AFF3B003C803D00F8
:10C000003E003F004040410042004300447F45FF66
:10C0100046FF4700480049004A004B004C034DC012
:10C020004E004F00500B5140520053000098080042
:10C0300009000A000B000C000D000E000F0010009C
:10C040001110120013001400151016041701180027
:10C0500019601A281B001C001D701E2C1F012000D7
:10C0600021002200230024002500260027002800AC
:10C0700029402A002B022C002D602E382F02300080
:10C08000316032083305340135B0360437043800E6
:10C0900039403A043B033C003D703E003F03400101
:10C0A00041B0420C43074400457046104708480021
:10C0B00049004A004B004C004D004E004F0050001C
:10C0C00051405200530654005560563857065800E8
:10C0D00059605A1C5B0B5C015DB05E185F0A600022
:10C0E0006140620463096400657066146709680151
:10C0F00069B06A206B0D6C006D706E246F0E70005D
:10C10000710072007300740075007600770078008B
:10C1100079407A007B0C7C007D607E387F0C009932
:10C12000080009600A380B0C0C000D000E000F000F
:10C13000100011401204131814001540160417368D
:10C14000180019601A471BFB1C001D001E001F0071
:10C1500020002100220023002400253026F02702A1
:10C16000280129142A832B772C002D002E002F0064
:10C1700030003160324B33FB34003500360037007D
:10C18000380039003A003B003C003D303EF03F02B1
:10C190004001411442834377440045004600470074
:10C1A0004800496F4AEC4B0F4C004D6F4EEC4F105E
:10C1B000500051305200530254005530560057027F
:10C1C0005800596F5AEC5B115C005D6F5EEC5F12BA
:10C1D00060006130620063026400653066006702DF
:10C1E0006800696F6AEC6B136C006D6F6EEC6F1416
:10C1F000700071307200730274007530760077023F
:10C200007800796F7AEC7B157C007D6F7EEC7F1671
:10C21000009A080009300A000B020C000D300E00D5
:10C220000F021000116F12F0132D1400156F16F08D
:10C23000172E180019301A041B021C001D301E0492
:10C240001F022000216F22F0232F2400256F26F0EB
:10C250002730280029302A042B022C002D302E04F0
:10C260002F023000316F32F033313400356F36F049
:10C270003732380039303A043B023C003D303E044E
:10C280003F024000416F42F043334400456F46F0A7
:10C290004734480049304A044B024C004D304E04AC
:10C2A0004F0250015110520353FF00002B1F002C6E
:10C2B0000400010400000200080453070300FFFF0C
:10C2C000000000010304000003110210002C08000C
:10C2D00009000A200B000C000D000E200F001000BA
:10C2E000110012201300147F15B316781700188060
:10C2F00019981A861B001C001D001E201F0020001C
:10C300002100222023002400250026202700287F4A
:10C3100029B32A782B002C802D982E862F003040B0
:10C32000310032003300344035003600370038FF2A
:10C3300039FF3AFF3B003C803D003E003F0040405B
:10C34000410042004300447F45FF46FF470048004C
:10C3500049004A004B004C034DC04E004F00500BAB
:10C36000514052005300003E080009000A200B0013
:10C370000C000D000E200F00100011001220130001
:10C38000147F15B316781700188019981A861B00A9
:10C390001C001D001E201F00200021002220230061
:10C3A0002400250026202700287F29B32A782B0087
:10C3B0002C802D982E862F00304031003200330023
:10C3C000344035003600370038FF39FF3AFF3B0074
:10C3D0003C803D003E003F004040410042004300A1
:10C3E000447F45FF46FF4700480049004A004B0094
:10C3F0004C034DC04E004F00500B514052005300B3
:10C400000098080009000A000B000C000D000E0047
:10C410000F00100011101200130014001510160464
:10C420001701180019601A281B001C001D701E2C13
:10C430001F012000210022002300240025002600E7
:10C440002700280029402A002B022C002D602E38BE
:10C450002F023000316032083305340135B0360424
:10C460003704380039403A043B033C003D703E003D
:10C470003F03400141B0420C430744004570461061
:10C480004708480049004A004B004C004D004E0050
:10C490004F0050005140520053065400556056382A
:10C4A0005706580059605A1C5B0B5C015DB05E1862
:10C4B0005F0A60006140620463096400657066148D
:10C4C0006709680169B06A206B0D6C006D706E249D
:10C4D0006F0E7000710072007300740075007600BA
:10C4E0007700780079407A007B0C7C007D607E3894
:10C4F0007F0C0099080009600A380B0C0C000D0035
:10C500000E000F0010001140120413181400154003
:10C5100016041736180019601A471BFB1C001D0073
:10C520001E001F00200021002200230024002530CF
:10C5300026F02702280129142A832B772C002D00AE
:10C540002E002F0030003160324B33FB34003500B9
:10C5500036003700380039003A003B003C003D30DF
:10C560003EF03F02400141144283437744004500BE
:10C57000460047004800496F4AEC4B0F4C004D6F96
:10C580004EEC4F10500051305200530254005530C1
:10C59000560057025800596F5AEC5B115C005D6FF2
:10C5A0005EEC5F126000613062006302640065301F
:10C5B000660067026800696F6AEC6B136C006D6F50
:10C5C0006EEC6F147000713072007302740075307D
:10C5D000760077027800796F7AEC7B157C007D6FAE
:10C5E0007EEC7F16009A080009300A000B020C004E
:10C5F0000D300E000F021000116F12F0132D1400F9
:10C60000156F16F0172E180019301A041B021C00A3
:10C610001D301E041F022000216F22F0232F240052
:10C62000256F26F02730280029302A042B022C0001
:10C630002D302E042F023000316F32F033313400B0
:10C64000356F36F03732380039303A043B023C005F
:10C650003D303E043F024000416F42F0433344000E
:10C66000456F46F04734480049304A044B024C00BD
:10C670004D304E044F0250015110520353FF000041
:10C680002B1F002C040001040000020008045307C3
:10C690000300FFFF0000000103040000031102106B
:10C6A000002C080009030A620B000C000D030E6247
:10C6B0000F001000110312621300147E156E165144
:10C6C0001700188319151A031B001C001D031E6296
:10C6D0001F0020002103226223002400250326627C
:10C6E0002700287E296E2A512B002C832D152E031E
:10C6F0002F00304031003200330034403500360026
:10C70000370038FF39FF3AFF3B003C803D003E00D8
:10C710003F004040410042004300447F45FF46FF48
:10C720004700480049004A004B004C034DC04E00F2
:10C730004F00500B514052005300003E08000903C7
:10C740000A620B000C000D030E620F0010001103B3
:10C7500012621300147E156E1651170018831915F6
:10C760001A031B001C001D031E621F002000210372
:10C77000226223002400250326622700287E296EDA
:10C780002A512B002C832D152E032F003040310011
:10C7900032003300344035003600370038FF39FFAF
:10C7A0003AFF3B003C803D003E003F0040404100DE
:10C7B00042004300447F45FF46FF470048004900D0
:10C7C0004A004B004C034DC04E004F00500B5140EF
:10C7D000520053000098080009000A000B000C00EA
:10C7E0000D000E000F0010001110120013001400B5
:10C7F000151016041701180019601A281B001C00D8
:10C800001D701E2C1F012000210022002300240087
:10C81000250026002700280029402A002B022C0092
:10C820002D602E382F02300031603208330534017C
:10C8300035B036043704380039403A043B033C0035
:10C840003D703E003F03400141B0420C43074400AD
:10C85000457046104708480049004A004B004C000C
:10C860004D004E004F0050005140520053065400FE
:10C87000556056385706580059605A1C5B0B5C01CE
:10C880005DB05E185F0A6000614062046309640085
:10C89000657066146709680169B06A206B0D6C00E9
:10C8A0006D706E246F0E7000710072007300740062
:10C8B000750076007700780079407A007B0C7C0068
:10C8C0007D607E387F0C0099080009600A380B0CE7
:10C8D0000C000D000E000F00100011401204131880
:10C8E0001400154016041736180019601A471BFB70
:10C8F0001C001D001E001F0020002100220023003C
:10C900002400253026F02702280129142A832B77BA
:10C910002C002D002E002F0030003160324B33FBF5
:10C920003400350036003700380039003A003B004B
:10C930003C003D303EF03F024001411442834377CA
:10C9400044004500460047004800496F4AEC4B0F41
:10C950004C004D6F4EEC4F105000513052005302BE
:10C9600054005530560057025800596F5AEC5B116D
:10C970005C005D6F5EEC5F1260006130620063021C
:10C9800064006530660067026800696F6AEC6B13CB
:10C990006C006D6F6EEC6F1470007130720073027A
:10C9A00074007530760077027800796F7AEC7B1529
:10C9B0007C007D6F7EEC7F16009A080009300A002B
:10C9C0000B020C000D300E000F021000116F12F060
:10C9D000132D1400156F16F0172E180019301A04B5
:10C9E0001B021C001D301E041F022000216F22F0BC
:10C9F000232F2400256F26F02730280029302A0411
:10CA00002B022C002D302E042F023000316F32F01B
:10CA100033313400356F36F03732380039303A046C
:10CA20003B023C003D303E043F024000416F42F07B
:10CA300043334400456F46F04734480049304A04C8
:10CA40004B024C004D304E044F0250015110520326
:10CA500053FF00002B1F002C040001040000020003
:10CA6000080453070300FFFF000000010304000057
:10CA700003110210002C080009000AB80B000C007A
:10CA80000D000EB80F001000110012B81300147F33
:10CA90001548160C17001881196C1ADB1B001C00B6
:10CAA0001D001EB81F002000210022B82300240012
:10CAB000250026B82700287F29482A0C2B002C8126
:10CAC0002D6C2EDB2F00304031003200330034401B
:10CAD00035003600370038FF39FF3AFF3B003C8015
:10CAE0003D003E003F004040410042004300447F83
:10CAF00045FF46FF4700480049004A004B004C03F1
:10CB00004DC04E004F00500B514052005300003EAC
:10CB1000080009000AB80B000C000D000EB80F0049
:10CB20001000110012B81300147F1548160C1700DE
:10CB30001881196C1ADB1B001C001D001EB81F0099
:10CB40002000210022B823002400250026B8270059
:10CB5000287F29482A0C2B002C812D6C2EDB2F00DE
:10CB600030403100320033003440350036003700A9
:10CB700038FF39FF3AFF3B003C803D003E003F005C
:10CB80004040410042004300447F45FF46FF4700CC
:10CB9000480049004A004B004C034DC04E004F0076
:10CBA000500B5140520053000098080009000A0041
:10CBB0000B000C000D000E000F00100011101200F1
:10CBC00013001400151016041701180019601A2814
:10CBD0001B001C001D701E2C1F01200021002200C4
:10CBE00023002400250026002700280029402A00D1
:10CBF0002B022C002D602E382F02300031603208BD
:10CC00003305340135B036043704380039403A046E
:10CC10003B033C003D703E003F03400141B0420CED
:10CC200043074400457046104708480049004A0041
:10CC30004B004C004D004E004F0050005140520040
:10CC400053065400556056385706580059605A1C10
:10CC50005B0B5C015DB05E185F0A600061406204BE
:10CC600063096400657066146709680169B06A2029
:10CC70006B0D6C006D706E246F0E70007100720091
:10CC800073007400750076007700780079407A00B0
:10CC90007B0C7C007D607E387F0C00990800096069
:10CCA0000A380B0C0C000D000E000F001000114094
:10CCB00012041318140015401604173618001960D2
:10CCC0001A471BFB1C001D001E001F002000210036
:10CCD000220023002400253026F0270228012914F1
:10CCE0002A832B772C002D002E002F00300031607E
:10CCF000324B33FB34003500360037003800390042
:10CD00003A003B003C003D303EF03F024001411400
:10CD10004283437744004500460047004800496F7E
:10CD20004AEC4B0F4C004D6F4EEC4F105000513001
:10CD30005200530254005530560057025800596FA4
:10CD40005AEC5B115C005D6F5EEC5F12600061305D
:10CD50006200630264006530660067026800696F04
:10CD60006AEC6B136C006D6F6EEC6F1470007130B9
:10CD70007200730274007530760077027800796F64
:10CD80007AEC7B157C007D6F7EEC7F16009A0800A4
:10CD900009300A000B020C000D300E000F021000CB
:10CDA000116F12F0132D1400156F16F0172E1800C6
:10CDB00019301A041B021C001D301E041F02200023
:10CDC000216F22F0232F2400256F26F02730280022
:10CDD00029302A042B022C002D302E042F02300083
:10CDE000316F32F033313400356F36F0373238007E
:10CDF00039303A043B023C003D303E043F024000E3
:10CE0000416F42F043334400456F46F047344800D9
:10CE100049304A044B024C004D304E044F02500141
:10CE20005110520353FF00002B1F002C040001047B
:10CE300000000200080453070300FFFF0000000188
:10CE40000304000003110210002C080009000A2E40
:10CE50000B000C000D000E2E0F0010001100122E02
:10CE60001300147F15A416251700188019B61AF19F
:10CE70001B001C001D001E2E1F0020002100222E62
:10CE8000230024002500262E2700287F29A42A25F8
:10CE90002B002C802DB62EF12F00304031003200B7
:10CEA0003300344035003600370038FF39FF3AFF91
:10CEB0003B003C803D003E003F00404041004200BE
:10CEC0004300447F45FF46FF4700480049004A00B1
:10CED0004B004C034DC04E004F00500B51405200D0
:10CEE0005300003E080009000A2E0B000C000D0044
:10CEF0000E2E0F0010001100122E1300147F15A427
:10CF000016251700188019B61AF11B001C001D0009
:10CF10001E2E1F0020002100222E230024002500A9
:10CF2000262E2700287F29A42A252B002C802DB609
:10CF30002EF12F00304031003200330034403500F4
:10CF40003600370038FF39FF3AFF3B003C803D0098
:10CF50003E003F004040410042004300447F45FF07
:10CF600046FF4700480049004A004B004C034DC0B3
:10CF70004E004F00500B51405200530000980800E3
:10CF800009000A000B000C000D000E000F0010003D
:10CF900011101200130014001510160417011800C8
:10CFA00019601A281B001C001D701E2C1F01200078
:10CFB000210022002300240025002600270028004D
:10CFC00029402A002B022C002D602E382F02300021
:10CFD000316032083305340135B036043704380087
:10CFE00039403A043B033C003D703E003F034001A2
:10CFF00041B0420C430744004570461047084800C2
:10D0000049004A004B004C004D004E004F005000BC
:10D010005140520053065400556056385706580088
:10D0200059605A1C5B0B5C015DB05E185F0A6000C2
:10D0300061406204630964006570661467096801F1
:10D0400069B06A206B0D6C006D706E246F0E7000FD
:10D05000710072007300740075007600770078002C
:10D0600079407A007B0C7C007D607E387F0C0099D3
:10D07000080009600A380B0C0C000D000E000F00B0
:10D08000100011401204131814001540160417362E
:10D09000180019601A471BFB1C001D001E001F0012
:10D0A00020002100220023002400253026F0270242
:10D0B000280129142A832B772C002D002E002F0005
:10D0C00030003160324B33FB34003500360037001E
:10D0D000380039003A003B003C003D303EF03F0252
:10D0E0004001411442834377440045004600470015
:10D0F0004800496F4AEC4B0F4C004D6F4EEC4F10FF
:10D10000500051305200530254005530560057021F
:10D110005800596F5AEC5B115C005D6F5EEC5F125A
:10D12000600061306200630264006530660067027F
:10D130006800696F6AEC6B136C006D6F6EEC6F14B6
:10D1400070007130720073027400753076007702DF
:10D150007800796F7AEC7B157C007D6F7EEC7F1612
:10D16000009A080009300A000B020C000D300E0076
:10D170000F021000116F12F0132D1400156F16F02E
:10D18000172E180019301A041B021C001D301E0433
:10D190001F022000216F22F0232F2400256F26F08C
:10D1A0002730280029302A042B022C002D302E0491
:10D1B0002F023000316F32F033313400356F36F0EA
:10D1C0003732380039303A043B023C003D303E04EF
:10D1D0003F024000416F42F043334400456F46F048
:10D1E0004734480049304A044B024C004D304E044D
:10D1F0004F0250015110520353FF00002B1F002C0F
:10D200000400010400000200080453070300FFFFAC
:10D21000000000010304000003110210002C0800AC
:10D2200009050A460B000C000D050E460F00100004
:10D23000110512461300147E1509163217001883C3
:10D2400019D71A411B001C001D051E461F00200097
:10D250002105224623002400250526462700287E96
:10D2600029092A322B002C832DD72E412F00304044
:10D27000310032003300344035003600370038FFCB
:10D2800039FF3AFF3B003C803D003E003F004040FC
:10D29000410042004300447F45FF46FF47004800ED
:10D2A00049004A004B004C034DC04E004F00500B4C
:10D2B000514052005300003E080009050A460B0089
:10D2C0000C000D050E460F0010001105124613004C
:10D2D000147E150916321700188319D71A411B003E
:10D2E0001C001D051E461F002000210522462300AC
:10D2F0002400250526462700287E29092A322B00EE
:10D300002C832DD72E412F003040310032003300C6
:10D31000344035003600370038FF39FF3AFF3B0014
:10D320003C803D003E003F00404041004200430041
:10D33000447F45FF46FF4700480049004A004B0034
:10D340004C034DC04E004F00500B51405200530053
:10D350000098080009000A000B000C000D000E00E8
:10D360000F00100011101200130014001510160405
:10D370001701180019601A281B001C001D701E2CB4
:10D380001F01200021002200230024002500260088
:10D390002700280029402A002B022C002D602E385F
:10D3A0002F023000316032083305340135B03604C5
:10D3B0003704380039403A043B033C003D703E00DE
:10D3C0003F03400141B0420C430744004570461002
:10D3D0004708480049004A004B004C004D004E00F1
:10D3E0004F005000514052005306540055605638CB
:10D3F0005706580059605A1C5B0B5C015DB05E1803
:10D400005F0A60006140620463096400657066142D
:10D410006709680169B06A206B0D6C006D706E243D
:10D420006F0E70007100720073007400750076005A
:10D430007700780079407A007B0C7C007D607E3834
:10D440007F0C0099080009600A380B0C0C000D00D5
:10D450000E000F00100011401204131814001540A4
:10D4600016041736180019601A471BFB1C001D0014
:10D470001E001F0020002100220023002400253070
:10D4800026F02702280129142A832B772C002D004F
:10D490002E002F0030003160324B33FB340035005A
:10D4A00036003700380039003A003B003C003D3080
:10D4B0003EF03F024001411442834377440045005F
:10D4C000460047004800496F4AEC4B0F4C004D6F37
:10D4D0004EEC4F1050005130520053025400553062
:10D4E000560057025800596F5AEC5B115C005D6F93
:10D4F0005EEC5F12600061306200630264006530C0
:10D50000660067026800696F6AEC6B136C006D6FF0
:10D510006EEC6F147000713072007302740075301D
:10D52000760077027800796F7AEC7B157C007D6F4E
:10D530007EEC7F16009A080009300A000B020C00EE
:10D540000D300E000F021000116F12F0132D140099
:10D55000156F16F0172E180019301A041B021C0044
:10D560001D301E041F022000216F22F0232F2400F3
:10D57000256F26F02730280029302A042B022C00A2
:10D580002D302E042F023000316F32F03331340051
:10D59000356F36F03732380039303A043B023C0000
:10D5A0003D303E043F024000416F42F043334400AF
:10D5B000456F46F04734480049304A044B024C005E
:10D5C0004D304E044F0250015110520353FF0000E2
:10D5D0002B1F002C04000104000002000804530764
:10D5E0000300FFFF0000000103040000031102100C
:10D5F000002C080009010A1F0B000C000D010E1F72
:10D600000F0010001101121F1300147F151916E8E6
:10D610001700188119C71A6E1B001C001D011E1F60
:10D620001F0020002101221F230024002501261FA6
:10D630002700287F29192AE82B002C812DC72E6E60
:10D640002F003040310032003300344035003600C6
:10D65000370038FF39FF3AFF3B003C803D003E0079
:10D660003F004040410042004300447F45FF46FFE9
:10D670004700480049004A004B004C034DC04E0093
:10D680004F00500B514052005300003E080009016A
:10D690000A1F0B000C000D010E1F0F0010001101DE
:10D6A000121F1300147F151916E81700188119C7E7
:10D6B0001A6E1B001C001D011E1F1F0020002101EF
:10D6C000221F230024002501261F2700287F291957
:10D6D0002AE82B002C812DC72E6E2F003040310000
:10D6E00032003300344035003600370038FF39FF50
:10D6F0003AFF3B003C803D003E003F00404041007F
:10D7000042004300447F45FF46FF47004800490070
:10D710004A004B004C034DC04E004F00500B51408F
:10D72000520053000098080009000A000B000C008A
:10D730000D000E000F001000111012001300140055
:10D74000151016041701180019601A281B001C0078
:10D750001D701E2C1F012000210022002300240028
:10D76000250026002700280029402A002B022C0033
:10D770002D602E382F02300031603208330534011D
:10D7800035B036043704380039403A043B033C00D6
:10D790003D703E003F03400141B0420C430744004E
:10D7A000457046104708480049004A004B004C00AD
:10D7B0004D004E004F00500051405200530654009F
:10D7C000556056385706580059605A1C5B0B5C016F
:10D7D0005DB05E185F0A6000614062046309640026
:10D7E000657066146709680169B06A206B0D6C008A
:10D7F0006D706E246F0E7000710072007300740003
:10D80000750076007700780079407A007B0C7C0008
:10D810007D607E387F0C0099080009600A380B0C87
:10D820000C000D000E000F00100011401204131820
:10D830001400154016041736180019601A471BFB10
:10D840001C001D001E001F002000210022002300DC
:10D850002400253026F02702280129142A832B775B
:10D860002C002D002E002F0030003160324B33FB96
:10D870003400350036003700380039003A003B00EC
:10D880003C003D303EF03F0240014114428343776B
:10D8900044004500460047004800496F4AEC4B0FE2
:10D8A0004C004D6F4EEC4F1050005130520053025F
:10D8B00054005530560057025800596F5AEC5B110E
:10D8C0005C005D6F5EEC5F126000613062006302BD
:10D8D00064006530660067026800696F6AEC6B136C
:10D8E0006C006D6F6EEC6F1470007130720073021B
:10D8F00074007530760077027800796F7AEC7B15CA
:10D900007C007D6F7EEC7F16009A080009300A00CB
:10D910000B020C000D300E000F021000116F12F000
:10D92000132D1400156F16F0172E180019301A0455
:10D930001B021C001D301E041F022000216F22F05C
:10D94000232F2400256F26F02730280029302A04B1
:10D950002B022C002D302E042F023000316F32F0BC
:10D9600033313400356F36F03732380039303A040D
:10D970003B023C003D303E043F024000416F42F01C
:10D9800043334400456F46F04734480049304A0469
:10D990004B024C004D304E044F02500151105203C7
:10D9A00053FF00002B1F002C0400010400000200A4
:10D9B000080453070300FFFF0000000103040000F8
:10D9C00003110210002C080009000A480B000C008B
:10D9D0000D000E480F001000110012481300147FB4
:10D9E000158D16251700188019E41A841B001C00D9
:10D9F0001D001E481F002000210022482300240093
:10DA0000250026482700287F298D2A252B002C80D9
:10DA10002DE42E842F00304031003200330034409A
:10DA200035003600370038FF39FF3AFF3B003C80B5
:10DA30003D003E003F004040410042004300447F23
:10DA400045FF46FF4700480049004A004B004C0391
:10DA50004DC04E004F00500B514052005300003E4D
:10DA6000080009000A480B000C000D000E480F00CA
:10DA70001000110012481300147F158D1625170091
:10DA8000188019E41A841B001C001D001E481F008A
:10DA900020002100224823002400250026482700DA
:10DAA000287F298D2A252B002C802DE42E842F0001
:10DAB000304031003200330034403500360037004A
:10DAC00038FF39FF3AFF3B003C803D003E003F00FD
:10DAD0004040410042004300447F45FF46FF47006D
:10DAE000480049004A004B004C034DC04E004F0017
:10DAF000500B5140520053000098080009000A00E2
:10DB00000B000C000D000E000F0010001110120091
:10DB100013001400151016041701180019601A28B4
:10DB20001B001C001D701E2C1F0120002100220064
:10DB300023002400250026002700280029402A0071
:10DB40002B022C002D602E382F023000316032085D
:10DB50003305340135B036043704380039403A040F
:10DB60003B033C003D703E003F03400141B0420C8E
:10DB700043074400457046104708480049004A00E2
:10DB80004B004C004D004E004F00500051405200E1
:10DB900053065400556056385706580059605A1CB1
:10DBA0005B0B5C015DB05E185F0A6000614062045F
:10DBB00063096400657066146709680169B06A20CA
:10DBC0006B0D6C006D706E246F0E70007100720032
:10DBD00073007400750076007700780079407A0051
:10DBE0007B0C7C007D607E387F0C0099080009600A
:10DBF0000A380B0C0C000D000E000F001000114035
:10DC00001204131814001540160417361800196072
:10DC10001A471BFB1C001D001E001F0020002100D6
:10DC2000220023002400253026F027022801291491
:10DC30002A832B772C002D002E002F00300031601E
:10DC4000324B33FB340035003600370038003900E2
:10DC50003A003B003C003D303EF03F0240014114A1
:10DC60004283437744004500460047004800496F1F
:10DC70004AEC4B0F4C004D6F4EEC4F1050005130A2
:10DC80005200530254005530560057025800596F45
:10DC90005AEC5B115C005D6F5EEC5F1260006130FE
:10DCA0006200630264006530660067026800696FA5
:10DCB0006AEC6B136C006D6F6EEC6F14700071305A
:10DCC0007200730274007530760077027800796F05
:10DCD0007AEC7B157C007D6F7EEC7F16009A080045
:10DCE00009300A000B020C000D300E000F0210006C
:10DCF000116F12F0132D1400156F16F0172E180067
:10DD000019301A041B021C001D301E041F022000C3
:10DD1000216F22F0232F2400256F26F027302800C2
:10DD200029302A042B022C002D302E042F02300023
:10DD3000316F32F033313400356F36F0373238001E
:10DD400039303A043B023C003D303E043F02400083
:10DD5000416F42F043334400456F46F0473448007A
:10DD600049304A044B024C004D304E044F025001E2
:10DD70005110520353FF00002B1F002C040001041C
:10DD800000000200080453070300FFFF0000000129
:10DD90000304000003110210002C080009090A54B2
:10DDA0000B000C000D090E540F0010001109125445
:10DDB0001300147D1560160F1700188519181A59CD
:10DDC0001B001C001D091E541F00200021092254A5
:10DDD00023002400250926542700287D29602A0FC6
:10DDE0002B002C852D182E592F0030403100320089
:10DDF0003300344035003600370038FF39FF3AFF32
:10DE00003B003C803D003E003F004040410042005E
:10DE10004300447F45FF46FF4700480049004A0051
:10DE20004B004C034DC04E004F00500B5140520070
:10DE30005300003E080009090A540B000C000D09AC
:10DE40000E540F001000110912541300147D1560B8
:10DE5000160F1700188519181A591B001C001D09E8
:10DE60001E541F00200021092254230024002509EC
:10DE700026542700287D29602A0F2B002C852D1879
:10DE80002E592F003040310032003300344035002D
:10DE90003600370038FF39FF3AFF3B003C803D0039
:10DEA0003E003F004040410042004300447F45FFA8
:10DEB00046FF4700480049004A004B004C034DC054
:10DEC0004E004F00500B5140520053000098080084
:10DED00009000A000B000C000D000E000F001000DE
:10DEE0001110120013001400151016041701180069
:10DEF00019601A281B001C001D701E2C1F01200019
:10DF000021002200230024002500260027002800ED
:10DF100029402A002B022C002D602E382F023000C1
:10DF2000316032083305340135B036043704380027
:10DF300039403A043B033C003D703E003F03400142
:10DF400041B0420C43074400457046104708480062
:10DF500049004A004B004C004D004E004F0050005D
:10DF60005140520053065400556056385706580029
:10DF700059605A1C5B0B5C015DB05E185F0A600063
:10DF80006140620463096400657066146709680192
:10DF900069B06A206B0D6C006D706E246F0E70009E
:10DFA00071007200730074007500760077007800CD
:10DFB00079407A007B0C7C007D607E387F0C009974
:10DFC000080009600A380B0C0C000D000E000F0051
:10DFD00010001140120413181400154016041736CF
:10DFE000180019601A471BFB1C001D001E001F00B3
:10DFF00020002100220023002400253026F02702E3
:10E00000280129142A832B772C002D002E002F00A5
:10E0100030003160324B33FB3400350036003700BE
:10E02000380039003A003B003C003D303EF03F02F2
:10E0300040014114428343774400450046004700B5
:10E040004800496F4AEC4B0F4C004D6F4EEC4F109F
:10E0500050005130520053025400553056005702C0
:10E060005800596F5AEC5B115C005D6F5EEC5F12FB
:10E070006000613062006302640065306600670220
:10E080006800696F6AEC6B136C006D6F6EEC6F1457
:10E090007000713072007302740075307600770280
:10E0A0007800796F7AEC7B157C007D6F7EEC7F16B3
:10E0B000009A080009300A000B020C000D300E0017
:10E0C0000F021000116F12F0132D1400156F16F0CF
:10E0D000172E180019301A041B021C001D301E04D4
:10E0E0001F022000216F22F0232F2400256F26F02D
:10E0F0002730280029302A042B022C002D302E0432
:10E100002F023000316F32F033313400356F36F08A
:10E110003732380039303A043B023C003D303E048F
:10E120003F024000416F42F043334400456F46F0E8
:10E130004734480049304A044B024C004D304E04ED
:10E140004F0250015110520353FF00002B1F002CAF
:10E150000400010400000200080453070300FFFF4D
:10E16000000000010304000003110210002C08004D
:10E1700009010AFD0B000C000D010EFD0F0010003F
:10E18000110112FD1300147E15CC16DF1700188242
:10E19000195D1AD21B001C001D011EFD1F0020006E
:10E1A000210122FD23002400250126FD2700287ED1
:10E1B00029CC2ADF2B002C822D5D2ED22F0030405F
:10E1C000310032003300344035003600370038FF6C
:10E1D00039FF3AFF3B003C803D003E003F0040409D
:10E1E000410042004300447F45FF46FF470048008E
:10E1F00049004A004B004C034DC04E004F00500BED
:10E20000514052005300003E080009010AFD0B0076
:10E210000C000D010EFD0F001000110112FD130086
:10E22000147E15CC16DF17001882195D1AD21B0058
:10E230001C001D011EFD1F002000210122FD2300E6
:10E240002400250126FD2700287E29CC2ADF2B006B
:10E250002C822D5D2ED22F00304031003200330051
:10E26000344035003600370038FF39FF3AFF3B00B5
:10E270003C803D003E003F004040410042004300E2
:10E28000447F45FF46FF4700480049004A004B00D5
:10E290004C034DC04E004F00500B514052005300F4
:10E2A0000098080009000A000B000C000D000E0089
:10E2B0000F001000111012001300140015101604A6
:10E2C0001701180019601A281B001C001D701E2C55
:10E2D0001F01200021002200230024002500260029
:10E2E0002700280029402A002B022C002D602E3800
:10E2F0002F023000316032083305340135B0360466
:10E300003704380039403A043B033C003D703E007E
:10E310003F03400141B0420C4307440045704610A2
:10E320004708480049004A004B004C004D004E0091
:10E330004F0050005140520053065400556056386B
:10E340005706580059605A1C5B0B5C015DB05E18A3
:10E350005F0A6000614062046309640065706614CE
:10E360006709680169B06A206B0D6C006D706E24DE
:10E370006F0E7000710072007300740075007600FB
:10E380007700780079407A007B0C7C007D607E38D5
:10E390007F0C0099080009600A380B0C0C000D0076
:10E3A0000E000F0010001140120413181400154045
:10E3B00016041736180019601A471BFB1C001D00B5
:10E3C0001E001F0020002100220023002400253011
:10E3D00026F02702280129142A832B772C002D00F0
:10E3E0002E002F0030003160324B33FB34003500FB
:10E3F00036003700380039003A003B003C003D3021
:10E400003EF03F02400141144283437744004500FF
:10E41000460047004800496F4AEC4B0F4C004D6FD7
:10E420004EEC4F1050005130520053025400553002
:10E43000560057025800596F5AEC5B115C005D6F33
:10E440005EEC5F1260006130620063026400653060
:10E45000660067026800696F6AEC6B136C006D6F91
:10E460006EEC6F14700071307200730274007530BE
:10E47000760077027800796F7AEC7B157C007D6FEF
:10E480007EEC7F16009A080009300A000B020C008F
:10E490000D300E000F021000116F12F0132D14003A
:10E4A000156F16F0172E180019301A041B021C00E5
:10E4B0001D301E041F022000216F22F0232F240094
:10E4C000256F26F02730280029302A042B022C0043
:10E4D0002D302E042F023000316F32F033313400F2
:10E4E000356F36F03732380039303A043B023C00A1
:10E4F0003D303E043F024000416F42F04333440050
:10E50000456F46F04734480049304A044B024C00FE
:10E510004D304E044F0250015110520353FF000082
:10E520002B1F002C04000104000002000804530704
:10E530000300FFFF000000010304000003110210AC
:10E54000002C080009000A7F0B000C000D000E7F54
:10E550000F0010001100127F1300147F156616C6FD
:10E560001700188119301A551B001C001D001E7F52
:10E570001F0020002100227F230024002500267F89
:10E580002700287F29662AC62B002C812D302E5586
:10E590002F00304031003200330034403500360067
:10E5A000370038FF39FF3AFF3B003C803D003E001A
:10E5B0003F004040410042004300447F45FF46FF8A
:10E5C0004700480049004A004B004C034DC04E0034
:10E5D0004F00500B514052005300003E080009000C
:10E5E0000A7F0B000C000D000E7F0F0010001100C1
:10E5F000127F1300147F156616C617001881193094
:10E600001A551B001C001D001E7F1F00200021004A
:10E61000227F230024002500267F2700287F2966EB
:10E620002AC62B002C812D302E552F003040310072
:10E6300032003300344035003600370038FF39FFF0
:10E640003AFF3B003C803D003E003F00404041001F
:10E6500042004300447F45FF46FF47004800490011
:10E660004A004B004C034DC04E004F00500B514030
:10E67000520053000098080009000A000B000C002B
:10E680000D000E000F0010001110120013001400F6
:10E69000151016041701180019601A281B001C0019
:10E6A0001D701E2C1F0120002100220023002400C9
:10E6B000250026002700280029402A002B022C00D4
:10E6C0002D602E382F0230003160320833053401BE
:10E6D00035B036043704380039403A043B033C0077
:10E6E0003D703E003F03400141B0420C43074400EF
:10E6F000457046104708480049004A004B004C004E
:10E700004D004E004F00500051405200530654003F
:10E71000556056385706580059605A1C5B0B5C010F
:10E720005DB05E185F0A60006140620463096400C6
:10E73000657066146709680169B06A206B0D6C002A
:10E740006D706E246F0E70007100720073007400A3
:10E75000750076007700780079407A007B0C7C00A9
:10E760007D607E387F0C0099080009600A380B0C28
:10E770000C000D000E000F001000114012041318C1
:10E780001400154016041736180019601A471BFBB1
:10E790001C001D001E001F0020002100220023007D
:10E7A0002400253026F02702280129142A832B77FC
:10E7B0002C002D002E002F0030003160324B33FB37
:10E7C0003400350036003700380039003A003B008D
:10E7D0003C003D303EF03F0240014114428343770C
:10E7E00044004500460047004800496F4AEC4B0F83
:10E7F0004C004D6F4EEC4F10500051305200530200
:10E8000054005530560057025800596F5AEC5B11AE
:10E810005C005D6F5EEC5F1260006130620063025D
:10E8200064006530660067026800696F6AEC6B130C
:10E830006C006D6F6EEC6F147000713072007302BB
:10E8400074007530760077027800796F7AEC7B156A
:10E850007C007D6F7EEC7F16009A080009300A006C
:10E860000B020C000D300E000F021000116F12F0A1
:10E87000132D1400156F16F0172E180019301A04F6
:10E880001B021C001D301E041F022000216F22F0FD
:10E89000232F2400256F26F02730280029302A0452
:10E8A0002B022C002D302E042F023000316F32F05D
:10E8B00033313400356F36F03732380039303A04AE
:10E8C0003B023C003D303E043F024000416F42F0BD
:10E8D00043334400456F46F04734480049304A040A
:10E8E0004B024C004D304E044F0250015110520368
:10E8F00053FF00002B1F002C040001040000020045
:10E90000080453070300FFFF000000010304000098
:10E9100003110210002C0800090E0A810B000C00E4
:10E920000D0E0E810F001000110E12811300147CC9
:10E9300015B616321700188619561A261B001C0029
:10E940001D0E1E811F002000210E228123002400A5
:10E95000250E26812700287C29B62A322B002C86FA
:10E960002D562E262F003040310032003300344027
:10E9700035003600370038FF39FF3AFF3B003C8056
:10E980003D003E003F004040410042004300447FC4
:10E9900045FF46FF4700480049004A004B004C0332
:10E9A0004DC04E004F00500B514052005300003EEE
:10E9B0000800090E0A810B000C000D0E0E810F00DD
:10E9C0001000110E12811300147C15B616321700B8
:10E9D000188619561A261B001C001D0E1E811F00CA
:10E9E0002000210E228123002400250E26812700ED
:10E9F000287C29B62A322B002C862D562E262F0055
:10EA000030403100320033003440350036003700EA
:10EA100038FF39FF3AFF3B003C803D003E003F009D
:10EA20004040410042004300447F45FF46FF47000D
:10EA3000480049004A004B004C034DC04E004F00B7
:10EA4000500B5140520053000098080009000A0082
:10EA50000B000C000D000E000F0010001110120032
:10EA600013001400151016041701180019601A2855
:10EA70001B001C001D701E2C1F0120002100220005
:10EA800023002400250026002700280029402A0012
:10EA90002B022C002D602E382F02300031603208FE
:10EAA0003305340135B036043704380039403A04B0
:10EAB0003B033C003D703E003F03400141B0420C2F
:10EAC00043074400457046104708480049004A0083
:10EAD0004B004C004D004E004F0050005140520082
:10EAE00053065400556056385706580059605A1C52
:10EAF0005B0B5C015DB05E185F0A60006140620400
:10EB000063096400657066146709680169B06A206A
:10EB10006B0D6C006D706E246F0E700071007200D2
:10EB200073007400750076007700780079407A00F1
:10EB30007B0C7C007D607E387F0C009908000960AA
:10EB40000A380B0C0C000D000E000F0010001140D5
:10EB50001204131814001540160417361800196013
:10EB60001A471BFB1C001D001E001F002000210077
:10EB7000220023002400253026F027022801291432
:10EB80002A832B772C002D002E002F0030003160BF
:10EB9000324B33FB34003500360037003800390083
:10EBA0003A003B003C003D303EF03F024001411442
:10EBB0004283437744004500460047004800496FC0
:10EBC0004AEC4B0F4C004D6F4EEC4F105000513043
:10EBD0005200530254005530560057025800596FE6
:10EBE0005AEC5B115C005D6F5EEC5F12600061309F
:10EBF0006200630264006530660067026800696F46
:10EC00006AEC6B136C006D6F6EEC6F1470007130FA
:10EC10007200730274007530760077027800796FA5
:10EC20007AEC7B157C007D6F7EEC7F16009A0800E5
:10EC300009300A000B020C000D300E000F0210000C
:10EC4000116F12F0132D1400156F16F0172E180007
:10EC500019301A041B021C001D301E041F02200064
:10EC6000216F22F0232F2400256F26F02730280063
:10EC700029302A042B022C002D302E042F023000C4
:10EC8000316F32F033313400356F36F037323800BF
:10EC900039303A043B023C003D303E043F02400024
:10ECA000416F42F043334400456F46F0473448001B
:10ECB00049304A044B024C004D304E044F02500183
:10ECC0005110520353FF00002B1F002C04000104BD
:10ECD00000000200080453070300FFFF00000001CA
:10ECE0000304000003110210002C080009030A1A93
:10ECF0000B000C000D030E1A0F0010001103121A66
:10ED00001300147E157F16AC1700188219F31A81B0
:10ED10001B001C001D031E1A1F0020002103221AC5
:10ED2000230024002503261A2700287E297F2AACE9
:10ED30002B002C822DF32E812F0030403100320029
:10ED40003300344035003600370038FF39FF3AFFD2
:10ED50003B003C803D003E003F00404041004200FF
:10ED60004300447F45FF46FF4700480049004A00F2
:10ED70004B004C034DC04E004F00500B5140520011
:10ED80005300003E080009030A1A0B000C000D0393
:10ED90000E1A0F0010001103121A1300147E157FB3
:10EDA00016AC1700188219F31A811B001C001D03F2
:10EDB0001E1A1F0020002103221A2300240025030D
:10EDC000261A2700287E297F2AAC2B002C822DF3BF
:10EDD0002E812F00304031003200330034403500A6
:10EDE0003600370038FF39FF3AFF3B003C803D00DA
:10EDF0003E003F004040410042004300447F45FF49
:10EE000046FF4700480049004A004B004C034DC0F4
:10EE10004E004F00500B5140520053000098080024
:10EE200009000A000B000C000D000E000F0010007E
:10EE30001110120013001400151016041701180009
:10EE400019601A281B001C001D701E2C1F012000B9
:10EE5000210022002300240025002600270028008E
:10EE600029402A002B022C002D602E382F02300062
:10EE7000316032083305340135B0360437043800C8
:10EE800039403A043B033C003D703E003F034001E3
:10EE900041B0420C43074400457046104708480003
:10EEA00049004A004B004C004D004E004F005000FE
:10EEB00051405200530654005560563857065800CA
:10EEC00059605A1C5B0B5C015DB05E185F0A600004
:10EED0006140620463096400657066146709680133
:10EEE00069B06A206B0D6C006D706E246F0E70003F
:10EEF000710072007300740075007600770078006E
:10EF000079407A007B0C7C007D607E387F0C009914
:10EF1000080009600A380B0C0C000D000E000F00F1
:10EF2000100011401204131814001540160417366F
:10EF3000180019601A471BFB1C001D001E001F0053
:10EF400020002100220023002400253026F0270283
:10EF5000280129142A832B772C002D002E002F0046
:10EF600030003160324B33FB34003500360037005F
:10EF7000380039003A003B003C003D303EF03F0293
:10EF80004001411442834377440045004600470056
:10EF90004800496F4AEC4B0F4C004D6F4EEC4F1040
:10EFA0005000513052005302540055305600570261
:10EFB0005800596F5AEC5B115C005D6F5EEC5F129C
:10EFC00060006130620063026400653066006702C1
:10EFD0006800696F6AEC6B136C006D6F6EEC6F14F8
:10EFE0007000713072007302740075307600770221
:10EFF0007800796F7AEC7B157C007D6F7EEC7F1654
:10F00000009A080009300A000B020C000D300E00B7
:10F010000F021000116F12F0132D1400156F16F06F
:10F02000172E180019301A041B021C001D301E0474
:10F030001F022000216F22F0232F2400256F26F0CD
:10F040002730280029302A042B022C002D302E04D2
:10F050002F023000316F32F033313400356F36F02B
:10F060003732380039303A043B023C003D303E0430
:10F070003F024000416F42F043334400456F46F089
:10F080004734480049304A044B024C004D304E048E
:10F090004F0250015110520353FF00002B1F002C50
:10F0A0000400010400000200080453070300FFFFEE
:10F0B000000000010304000003110210002C0800EE
:10F0C00009000AC70B000C000D000EC70F0010004E
:10F0D000110012C71300147F1540165C1700188129
:10F0E000197B1AF81B001C001D001EC71F00200002
:10F0F000210022C723002400250026C72700287FDF
:10F1000029402A5C2B002C812D7B2EF82F003040CB
:10F11000310032003300344035003600370038FF0C
:10F1200039FF3AFF3B003C803D003E003F0040403D
:10F13000410042004300447F45FF46FF470048002E
:10F1400049004A004B004C034DC04E004F00500B8D
:10F15000514052005300003E080009000AC70B004E
:10F160000C000D000EC70F001000110012C7130095
:10F17000147F1540165C17001881197B1AF81B00C4
:10F180001C001D001EC71F002000210022C72300F5
:10F190002400250026C72700287F29402A5C2B0051
:10F1A0002C812D7B2EF82F003040310032003300AF
:10F1B000344035003600370038FF39FF3AFF3B0056
:10F1C0003C803D003E003F00404041004200430083
:10F1D000447F45FF46FF4700480049004A004B0076
:10F1E0004C034DC04E004F00500B51405200530095
:10F1F0000098080009000A000B000C000D000E002A
:10F200000F00100011101200130014001510160446
:10F210001701180019601A281B001C001D701E2CF5
:10F220001F012000210022002300240025002600C9
:10F230002700280029402A002B022C002D602E38A0
:10F240002F023000316032083305340135B0360406
:10F250003704380039403A043B033C003D703E001F
:10F260003F03400141B0420C430744004570461043
:10F270004708480049004A004B004C004D004E0032
:10F280004F0050005140520053065400556056380C
:10F290005706580059605A1C5B0B5C015DB05E1844
:10F2A0005F0A60006140620463096400657066146F
:10F2B0006709680169B06A206B0D6C006D706E247F
:10F2C0006F0E70007100720073007400750076009C
:10F2D0007700780079407A007B0C7C007D607E3876
:10F2E0007F0C0099080009600A380B0C0C000D0017
:10F2F0000E000F00100011401204131814001540E6
:10F3000016041736180019601A471BFB1C001D0055
:10F310001E001F00200021002200230024002530B1
:10F3200026F02702280129142A832B772C002D0090
:10F330002E002F0030003160324B33FB340035009B
:10F3400036003700380039003A003B003C003D30C1
:10F350003EF03F02400141144283437744004500A0
:10F36000460047004800496F4AEC4B0F4C004D6F78
:10F370004EEC4F10500051305200530254005530A3
:10F38000560057025800596F5AEC5B115C005D6FD4
:10F390005EEC5F1260006130620063026400653001
:10F3A000660067026800696F6AEC6B136C006D6F32
:10F3B0006EEC6F147000713072007302740075305F
:10F3C000760077027800796F7AEC7B157C007D6F90
:10F3D0007EEC7F16009A080009300A000B020C0030
:10F3E0000D300E000F021000116F12F0132D1400DB
:10F3F000156F16F0172E180019301A041B021C0086
:10F400001D301E041F022000216F22F0232F240034
:10F41000256F26F02730280029302A042B022C00E3
:10F420002D302E042F023000316F32F03331340092
:10F43000356F36F03732380039303A043B023C0041
:10F440003D303E043F024000416F42F043334400F0
:10F45000456F46F04734480049304A044B024C009F
:10F460004D304E044F0250015110520353FF000023
:10F470002B1F002C040001040000020008045307A5
:10F480000300FFFF0000000103040000031102104D
:10F49000002C080009140AC80B000C000D140EC83B
:10F4A0000F001000111412C81300147C150B16A2C3
:10F4B0001700188719901AAD1B001C001D141EC8D8
:10F4C0001F002000211422C823002400251426C870
:10F4D0002700287C290B2AA22B002C872D902EADEB
:10F4E0002F00304031003200330034403500360008
:10F4F000370038FF39FF3AFF3B003C803D003E00BB
:10F500003F004040410042004300447F45FF46FF2A
:10F510004700480049004A004B004C034DC04E00D4
:10F520004F00500B514052005300003E0800091498
:10F530000AC80B000C000D140EC80F0010001114A7
:10F5400012C81300147C150B16A217001887199007
:10F550001AAD1B001C001D141EC81F002000211422
:10F5600022C823002400251426C82700287C290B44
:10F570002AA22B002C872D902EAD2F003040310079
:10F5800032003300344035003600370038FF39FF91
:10F590003AFF3B003C803D003E003F0040404100C0
:10F5A00042004300447F45FF46FF470048004900B2
:10F5B0004A004B004C034DC04E004F00500B5140D1
:10F5C000520053000098080009000A000B000C00CC
:10F5D0000D000E000F001000111012001300140097
:10F5E000151016041701180019601A281B001C00BA
:10F5F0001D701E2C1F01200021002200230024006A
:10F60000250026002700280029402A002B022C0074
:10F610002D602E382F02300031603208330534015E
:10F6200035B036043704380039403A043B033C0017
:10F630003D703E003F03400141B0420C430744008F
:10F64000457046104708480049004A004B004C00EE
:10F650004D004E004F0050005140520053065400E0
:10F66000556056385706580059605A1C5B0B5C01B0
:10F670005DB05E185F0A6000614062046309640067
:10F68000657066146709680169B06A206B0D6C00CB
:10F690006D706E246F0E7000710072007300740044
:10F6A000750076007700780079407A007B0C7C004A
:10F6B0007D607E387F0C0099080009600A380B0CC9
:10F6C0000C000D000E000F00100011401204131862
:10F6D0001400154016041736180019601A471BFB52
:10F6E0001C001D001E001F0020002100220023001E
:10F6F0002400253026F02702280129142A832B779D
:10F700002C002D002E002F0030003160324B33FBD7
:10F710003400350036003700380039003A003B002D
:10F720003C003D303EF03F024001411442834377AC
:10F7300044004500460047004800496F4AEC4B0F23
:10F740004C004D6F4EEC4F105000513052005302A0
:10F7500054005530560057025800596F5AEC5B114F
:10F760005C005D6F5EEC5F126000613062006302FE
:10F7700064006530660067026800696F6AEC6B13AD
:10F780006C006D6F6EEC6F1470007130720073025C
:10F7900074007530760077027800796F7AEC7B150B
:10F7A0007C007D6F7EEC7F16009A080009300A000D
:10F7B0000B020C000D300E000F021000116F12F042
:10F7C000132D1400156F16F0172E180019301A0497
:10F7D0001B021C001D301E041F022000216F22F09E
:10F7E000232F2400256F26F02730280029302A04F3
:10F7F0002B022C002D302E042F023000316F32F0FE
:10F8000033313400356F36F03732380039303A044E
:10F810003B023C003D303E043F024000416F42F05D
:10F8200043334400456F46F04734480049304A04AA
:10F830004B024C004D304E044F0250015110520308
:10F8400053FF00002B1F002C0400010400000200E5
:10F85000080453070300FFFF000000010304000039
:10F8600003110210002C080009040A750B000C009B
:10F870000D040E750F001000110412751300147E94
:10F880001532164F1700188319881A7D1B001C00AB
:10F890001D041E751F002000210422752300240072
:10F8A000250426752700287E29322A4F2B002C8319
:10F8B0002D882E7D2F00304031003200330034403F
:10F8C00035003600370038FF39FF3AFF3B003C80F7
:10F8D0003D003E003F004040410042004300447F65
:10F8E00045FF46FF4700480049004A004B004C03D3
:10F8F0004DC04E004F00500B514052005300003E8F
:10F90000080009040A750B000C000D040E750F00A9
:10F910001000110412751300147E1532164F1700D3
:10F92000188319881A7D1B001C001D041E751F00FA
:10F9300020002104227523002400250426752700B9
:10F94000287E29322A4F2B002C832D882E7D2F00D4
:10F95000304031003200330034403500360037008B
:10F9600038FF39FF3AFF3B003C803D003E003F003E
:10F970004040410042004300447F45FF46FF4700AE
:10F98000480049004A004B004C034DC04E004F0058
:10F99000500B5140520053000098080009000A0023
:10F9A0000B000C000D000E000F00100011101200D3
:10F9B00013001400151016041701180019601A28F6
:10F9C0001B001C001D701E2C1F01200021002200A6
:10F9D00023002400250026002700280029402A00B3
:10F9E0002B022C002D602E382F023000316032089F
:10F9F0003305340135B036043704380039403A0451
:10FA00003B033C003D703E003F03400141B0420CCF
:10FA100043074400457046104708480049004A0023
:10FA20004B004C004D004E004F0050005140520022
:10FA300053065400556056385706580059605A1CF2
:10FA40005B0B5C015DB05E185F0A600061406204A0
:10FA500063096400657066146709680169B06A200B
:10FA60006B0D6C006D706E246F0E70007100720073
:10FA700073007400750076007700780079407A0092
:10FA80007B0C7C007D607E387F0C0099080009604B
:10FA90000A380B0C0C000D000E000F001000114076
:10FAA00012041318140015401604173618001960B4
:10FAB0001A471BFB1C001D001E001F002000210018
:10FAC000220023002400253026F0270228012914D3
:10FAD0002A832B772C002D002E002F003000316060
:10FAE000324B33FB34003500360037003800390024
:10FAF0003A003B003C003D303EF03F0240014114E3
:10FB00004283437744004500460047004800496F60
:10FB10004AEC4B0F4C004D6F4EEC4F1050005130E3
:10FB20005200530254005530560057025800596F86
:10FB30005AEC5B115C005D6F5EEC5F12600061303F
:10FB40006200630264006530660067026800696FE6
:10FB50006AEC6B136C006D6F6EEC6F14700071309B
:10FB60007200730274007530760077027800796F46
:10FB70007AEC7B157C007D6F7EEC7F16009A080086
:10FB800009300A000B020C000D300E000F021000AD
:10FB9000116F12F0132D1400156F16F0172E1800A8
:10FBA00019301A041B021C001D301E041F02200005
:10FBB000216F22F0232F2400256F26F02730280004
:10FBC00029302A042B022C002D302E042F02300065
:10FBD000316F32F033313400356F36F03732380060
:10FBE00039303A043B023C003D303E043F024000C5
:10FBF000416F42F043334400456F46F047344800BC
:10FC000049304A044B024C004D304E044F02500123
:10FC10005110520353FF00002B1F002C040001045D
:10FC200000000200080453070300FFFF000000016A
:10FC30000304000003110210002C080009010A1F30
:10FC40000B000C000D010E1F0F0010001101121F00
:10FC50001300147F151916E81700188119C71A6EBA
:10FC60001B001C001D011E1F1F0020002101221F60
:10FC7000230024002501261F2700287F29192AE8B0
:10FC80002B002C812DC72E6E2F003040310032000A
:10FC90003300344035003600370038FF39FF3AFF73
:10FCA0003B003C803D003E003F00404041004200A0
:10FCB0004300447F45FF46FF4700480049004A0093
:10FCC0004B004C034DC04E004F00500B51405200B2
:10FCD0005300003E080009010A1F0B000C000D0133
:10FCE0000E1F0F0010001101121F1300147F1519B1
:10FCF00016E81700188119C71A6E1B001C001D0199
:10FD00001E1F1F0020002101221F230024002501A7
:10FD1000261F2700287F29192AE82B002C812DC7B0
:10FD20002E6E2F0030403100320033003440350059
:10FD30003600370038FF39FF3AFF3B003C803D007A
:10FD40003E003F004040410042004300447F45FFE9
:10FD500046FF4700480049004A004B004C034DC095
:10FD60004E004F00500B51405200530000980800C5
:10FD700009000A000B000C000D000E000F0010001F
:10FD800011101200130014001510160417011800AA
:10FD900019601A281B001C001D701E2C1F0120005A
:10FDA000210022002300240025002600270028002F
:10FDB00029402A002B022C002D602E382F02300003
:10FDC000316032083305340135B036043704380069
:10FDD00039403A043B033C003D703E003F03400184
:10FDE00041B0420C430744004570461047084800A4
:10FDF00049004A004B004C004D004E004F0050009F
:10FE0000514052005306540055605638570658006A
:10FE100059605A1C5B0B5C015DB05E185F0A6000A4
:10FE200061406204630964006570661467096801D3
:10FE300069B06A206B0D6C006D706E246F0E7000DF
:10FE4000710072007300740075007600770078000E
:10FE500079407A007B0C7C007D607E387F0C0099B5
:10FE6000080009600A380B0C0C000D000E000F0092
:10FE70001000114012041318140015401604173610
:10FE8000180019601A471BFB1C001D001E001F00F4
:10FE900020002100220023002400253026F0270224
:10FEA000280129142A832B772C002D002E002F00E7
:10FEB00030003160324B33FB340035003600370000
:10FEC000380039003A003B003C003D303EF03F0234
:10FED00040014114428343774400450046004700F7
:10FEE0004800496F4AEC4B0F4C004D6F4EEC4F10E1
:10FEF0005000513052005302540055305600570202
:10FF00005800596F5AEC5B115C005D6F5EEC5F123C
:10FF10006000613062006302640065306600670261
:10FF20006800696F6AEC6B136C006D6F6EEC6F1498
:10FF300070007130720073027400753076007702C1
:10FF40007800796F7AEC7B157C007D6F7EEC7F16F4
:10FF5000009A080009300A000B020C000D300E0058
:10FF60000F021000116F12F0132D1400156F16F010
:10FF7000172E180019301A041B021C001D301E0415
:10FF80001F022000216F22F0232F2400256F26F06E
:10FF90002730280029302A042B022C002D302E0473
:10FFA0002F023000316F32F033313400356F36F0CC
:10FFB0003732380039303A043B023C003D303E04D1
:10FFC0003F024000416F42F043334400456F46F02A
:10FFD0004734480049304A044B024C004D304E042F
:10FFE0004F0250015110520353FF00002B1F002CF1
:10FFF0000400010400000200080453070300FFFF8F
:020000040030CA
:0E00000000E8183C003F810000800FE00F4038
:00000001FF
